:1000000070C01895189518957AE04095089410F4EA
:10001000919802C0919A000013D012D046957A951B
:10002000B1F7089579E08099FECF0AD009D008D0C1
:100030008894809908947A9511F04795F7CF0895A0
:100040001CE31A95F1F708952FEF2A95F1F71A9509
:10005000D9F7089518E0331F10F4C59A01C0C59868
:10006000C79A0000C7981A95B1F7089518E030E0D4
:10007000330FB6993160C79A0000C7981A95C1F737
:100080000895C798BF9ABD9ABE98C49ABC9AC4985E
:100090001FEFDADF3CEADEDF33E5DCDFA0E2E6DF9C
:1000A000333559F030E0D6DFC79A0000C7983CEAF4
:1000B000D1DF33E5CFDFAA9591F730E0CBDF10E158
:1000C000C3DF089541E4A0DF46E59EDF42E59CDF03
:1000D00040E29ADF49E498DF43E596DF40E594DFAC
:1000E000089511271BBFC09AAFDFB09B09C0899844
:1000F000BF98BD98C598C798BC9810E315BF889560
:10010000C49ABC9AC498899A919A88988BDF4B318B
:10011000E9F3443519F486DF042FE6C0433511F4C2
:10012000D1DFF4CF463529F443E36EDF41E36CDFE2
:10013000EDCF463729F441E367DF41E365DFE6CFE2
:10014000443729F448E660DF40E05EDFDFCF403728
:1001500019F443E559DFDACF413619F449E554DFA4
:10016000D5CF483709F4C0C0493709F4BDC00836B7
:1001700009F0B7C0403511F484DFB6C0433481F4D0
:1001800051DF38E467DF362F65DF352F63DF342F2B
:1001900061DF10E259DF11E02227510F621FA4C076
:1001A000433661F43FDF30E455DF362F53DF352F20
:1001B00051DF342F4FDF10E247DF96C04235B9F4EC
:1001C00038E248DF362F46DF352F44DF4FDF432F3D
:1001D0001BDF30E23FDF362F3DDF352F3BDF46DFD1
:1001E000432F12DF11E02227510F621F8FCF4134BE
:1001F00029F418DF642F16DF542F76C0443481F4BD
:1002000011DF30EC27DF362F25DF352F23DF342FAA
:1002100021DF10E219DF11E02227510F621F64C0B5
:10022000443671F430EA16DF362F14DF352F12DF33
:100230001DDF432FE9DE11E02227510F621F66CF39
:100240004C3449F41FEF00DF1FEFFEDE1FEFFCDE32
:100250001FEFFADE49C0453659F43CEAFBDE30E8D0
:10026000F9DE34E0F7DE30E0F5DE10E3EDDE3CC031
:100270004C3671F4D7DE3CEAEDDE342F3670366E44
:10028000E9DE30E0E7DE30E0E5DE10E3DDDE2CC065
:10029000433789F4B2E005D0B1E003D0B0E001D03B
:1002A00035CF30E3D7DE30E0D5DE3B2FD3DEDEDEE8
:1002B000432FAADE08954A33A1F4B4DEC42FB2DE80
:1002C000D42FB0DEE42F03D01FEFBEDE0DC03C2FD5
:1002D000C1DE3D2FBFDE3E2FBDDEC8DE432F94DEE4
:1002E00008954FE391DE12CF4DE08EDE0FCFFFFF7A
:1002F000FFFFFFFFFFFFFFFFFFFFFFFFFFFFFFFF0E
:10030000FFFFFFFFFFFFFFFFFFFFFFFFFFFFFFFFFD
:10031000FFFFFFFFFFFFFFFFFFFFFFFFFFFFFFFFED
:10032000FFFFFFFFFFFFFFFFFFFFFFFFFFFFFFFFDD
:10033000FFFFFFFFFFFFFFFFFFFFFFFFFFFFFFFFCD
:10034000FFFFFFFFFFFFFFFFFFFFFFFFFFFFFFFFBD
:10035000FFFFFFFFFFFFFFFFFFFFFFFFFFFFFFFFAD
:10036000FFFFFFFFFFFFFFFFFFFFFFFFFFFFFFFF9D
:10037000FFFFFFFFFFFFFFFFFFFFFFFFFFFFFFFF8D
:10038000FFFFFFFFFFFFFFFFFFFFFFFFFFFFFFFF7D
:10039000FFFFFFFFFFFFFFFFFFFFFFFFFFFFFFFF6D
:1003A000FFFFFFFFFFFFFFFFFFFFFFFFFFFFFFFF5D
:1003B000FFFFFFFFFFFFFFFFFFFFFFFFFFFFFFFF4D
:1003C000FFFFFFFFFFFFFFFFFFFFFFFFFFFFFFFF3D
:1003D000FFFFFFFFFFFFFFFFFFFFFFFFFFFFFFFF2D
:1003E000FFFFFFFFFFFFFFFFFFFFFFFFFFFFFFFF1D
:1003F000FFFFFFFFFFFFFFFFFFFFFFFFFFFFFFFF0D
:00000001FF
